:080000000528000000000000CB
:0800080005288B138B1B052852
:100010002C2862088207022907290C298207473405
:100020002D34533443344F34503445342034203449
:10003000203452344134543445342034203456343E
:1000400050342D34503420342034203420342034A3
:100050002034203448345A34831203138313850127
:1000600086010F308700880189018316FF308500E3
:100070008600003087008801890106308100043045
:100080009F0083121F30870001309F00BB22103079
:10009000FB00C4229C30A022F8010030B9221030AD
:1000A000F200F101AB22F8010330B8220D30F2006A
:1000B000AB22F4218030ED001F1586188228E00164
:1000C000E1011F1961281E081F15E00BE10B6928CB
:1000D0008228723E031C61281F196C2878301E028A
:1000E0001F15E00BE10B7528822803186C281F19D7
:1000F00077281E091F15E00BE10B7F288228803E20
:10010000031C7728203084004030F4001F19862813
:100110001E091F158000840AF40B8628A030840075
:1001200074171F1991281E091F158000840AF40BEB
:100130009128F001F3012030F5008400000CEC0060
:100140006C0C3F39FC008030FE00B520F30AF31D33
:10015000A328A030F5008030FE00B520F30A731EFE
:10016000AB28ED1B0920E1215C287008750784008D
:10017000000CEC006C0C3F39EC00FD007C02031C11
:10018000C5287C08FD006C08FC00D0206C08FC0031
:10019000F00A70130310FE0C031CB528E5200800BC
:1001A000831720307C0784007C08F4007E088004DC
:1001B00074087D060319E3287E088004F40A741B82
:1001C000E328840AD8288313080020303F3E8400A7
:1001D0004030F4000230F8007308F7002122B030FC
:1001E000A0227022831700088001831384039122C8
:1001F000B230A022F403031908007B08F7070318A4
:10020000F80AEE284630E5005530E60010296E3039
:10021000E5004D30E60010298030E5001830E6009A
:100220001F15E301E4011F1913291E09E7001F151B
:1002300078306707031C1E2969141F29E9138830C9
:1002400067070318252969102629E9136908680634
:10025000E30703080139E4076908E800E50B1329FF
:10026000E60B132920308400FF30EA00EB018313F2
:100270003D21A03084003D214F294030F40000088A
:100280006A02031C45290008EA006B080002031CEF
:100290004B290008EB00840AF40B3F2908006A0888
:1002A0006B0283160317A200A401A3010310A20D81
:1002B000A30D982103138312F8010030B8222122E4
:1002C000B030A022273080388400831700088313C1
:1002D000103815222E30E03E1522840383170008C3
:1002E000831310381522B230A02263088316031737
:1002F000A20003138312640883160317A300A4014A
:10030000982103138312F8010930B8222122B0305A
:10031000A0222930803884000530F40083170008BB
:10032000831315228403F40B8E29B230A022080017
:1003300083179D21CA2183130800C1211830A00012
:10034000AD292530803884000730A10003308007B4
:10035000801D8002840AA10BA729BD212530803889
:1003600084000830A100800D001A03140012840AD2
:10037000A10BB329A00BA1290800A20DA30DA40D68
:100380000800A501A601A701A801A901AA01AB01C6
:10039000AC0108000830F0002C30803884000008E0
:1003A000031DDB292030E03E80008403F00BCF29C1
:1003B0001030A5040800103080048403F00BDB2902
:1003C0000800061CE8296D10061D012A6D110800A1
:1003D0006D18080040309F071F08C039C03A031D40
:1003E000F3291F139F136D141F0E0C39E200031025
:1003F000E20CE20CF8010F30B9226208103E0B2229
:1004000008006D1908008030ED079830ED1B9C3016
:10041000A0226D150800F9002122B030A022702220
:1004200079089122B230A0220800FA0082227A08CC
:100430009122080070227708912270227808912278
:1004400008007022770891227022780891222430C7
:10045000A0220800F801F7011A224030A02208006B
:100460000230F800F7011A224230A0220800F801F9
:100470007B08F7001A224130A0220800F8017B080F
:10048000F7001A224330A02208008030A022080082
:100490009C30A0220800F801F7012122B030A022F0
:1004A0000830F2007B08F10000301522F10B542ACD
:1004B000F20B522AB230A02208000230F800F701F5
:1004C0002122B030A0224030F2007B08F100003041
:1004D0001522F10B672AF20B652AB230A022080020
:1004E0008316FF3088008312193087000000081C33
:1004F000772A881C792A1F3087000000831688011C
:1005000083120800831688158312193087000000B3
:10051000881D882A1F3087000000831688118312E7
:100520000800FA00173087007A08880000001230AF
:10053000870000001730870000001F308700080088
:10054000FA0070227A08880000001A308700000044
:100550001F30870008002122B030A02271080E2031
:10056000E03E1522F10AF20BAE2AB230A0220800BA
:10057000703EF70008000530F6008B010B1DBE2A07
:100580000B11F60BBE2A08001F3087002A223022EA
:00000001FF
